:100000000C9462000C94D11A0C94FE1A0C948A0081
:100010000C948A000C948A000C948A000C948A0038
:100020000C948A000C948A000C948A000C948A0028
:100030000C948A000C94BC060C948A000C948A00E0
:100040000C942B1B0C948A000C947E1E0C94B91EED
:100050000C948A000C948A000C948A000C948A00F8
:100060000C9440050C948A00000000002400270036
:100070002A0000000000250028002B0000000000DE
:1000800023002600290004040404040404040202DA
:100090000202020203030303030301020408102007
:1000A0004080010204081020010204081020000012
:1000B0000007000201000003040600000000000029
:1000C0000000612011241FBECFEFD8E0DEBFCDBFFE
:1000D00012E0A0E0B1E0E8ECF2E402C005900D927D
:1000E000A43DB107D9F714E0A4EDB2E001C01D9220
:1000F000AE3BB107E1F710E0C4ECD0E004C02297BA
:10010000FE010E945E21C23CD107C9F70E94A620D1
:100110000C9462210C940000FB01DC0102C00190F0
:100120000D9241505040D8F708958091D40281300B
:1001300019F482E08093D4028091D402833019F4C0
:1001400084E08093D4020895E3E0F0E089E08093B6
:100150005700849190E08670863009F491E0892FF1
:1001600008951F93182F0E94A400882379F09FB749
:1001700081E080930404F894A89588E1809360005E
:1001800010936000112309F0A8959FBF1F91089557
:10019000382F20E080910504909106048227932750
:1001A00040E061E270E19C01220F331F97FF04C021
:1001B000C9018627972701C0C9014F5F483099F7C9
:1001C000909306048093050408958436910520F4E5
:1001D000BC0180E090E025C08E3B910550F48A552B
:1001E0009040BC0180E090E02AE030E040E050E048
:1001F00016C0823D910550F4845B9040BC0180E0C4
:1002000090E024E630E040E050E009C08D5C904092
:10021000BC0180E090E028E532E040E050E00E9440
:10022000B52024E630E040E050E00E94B52008957B
:1002300090E08C599F4F0E94E5000895DC0198964C
:10024000EC91F0E0E770F070E454FD4F8081089588
:10025000FC0120A530E0C9018170907001962770E3
:10026000307035952795820F931F880F880F08955A
:100270008F929F92AF92BF92CF92DF92EF92FF92B6
:100280000F931F938C010E941E01D80197962C9109
:1002900030E043E150E0249FF001259FF00D349FB2
:1002A000F00D1124E051FE4F80809180A280B38038
:1002B00090E00F96AA2797FDA095BA2FBC01CD011B
:1002C00020E43FE14DE750E00E94B520A5019401F4
:1002D0000E94E82069017A0180ED97E0A0E0B0E09B
:1002E000C80ED91EEA1EFB1ED80198968C91887103
:1002F00081F060E07EEE8AEB9BE0A50194010E9414
:10030000E82028513C4F4F4F5F4FC20ED31EE41ED2
:10031000F51E87EE93E0A0E0B0E0C80ED91EEA1EFD
:10032000FB1EC701B60128EE33E040E050E00E941A
:10033000E820CA01B90128EE33E040E050E00E9415
:10034000B5201F910F91FF90EF90DF90CF90BF905D
:10035000AF909F908F9008951F93182FDB01FA01A3
:10036000482F469530E0848190E083709070982FFC
:1003700088272081820F911D11969C938E938481F2
:1003800090E08C70907076E0880F991F7A95E1F775
:100390002181820F911D13969C938E9312978481D5
:1003A00090E08073907064E0880F991F6A95E1F780
:1003B0002281820F911D15969C938E9314978481B0
:1003C00090E0807C9070880F991F880F991F23817F
:1003D000820F911D17969C938E93169735961896BB
:1003E0003F5F431708F0BFCF10FF50C08081829558
:1003F00086958695837090E02DE431E0AC01429FB4
:10040000C001439F900D529F900D11240C961196A0
:100410009C938E93808190E044E0969587954A95D1
:10042000E1F783709070AC01429FC001439F900D33
:10043000529F900D11240C9613969C938E931297B5
:10044000808190E0969587959695879583709070BA
:10045000AC01429FC001439F900D529F900D11240B
:100460000C9615969C938E931497808190E08370E0
:100470009070AC01429FC001439F900D529F900D20
:1004800011240C9617969C938E9316971F9108959E
:1004900023E08032920718F420E030E026C023E009
:1004A000883E920748F49C012F51334054E0369522
:1004B00027955A95E1F719C027E0803D920720F46F
:1004C0009C012C5D334011C028E08839920718F058
:1004D0002FEF33E00AC09C01285C374044E036959A
:1004E00027954A95E1F72D503C4FC90108958C306E
:1004F000910548F49C0174E0220F331F7A95E1F7CF
:10050000285D3C4F17C023E0843F920720F49C01F4
:1005100024523C4F0FC024E08030920718F020E9AD
:1005200038E008C09C012657334F64E0220F331F88
:100530006A95E1F7C90108959C01369527952575BF
:100540003575821B930B9C0136952795369527951B
:100550002373337383739373280F391FC901E4E046
:1005600096958795EA95E1F7820F931F8F709F709C
:1005700021E031E0AC01429FC001439F900D529FAA
:10058000900D1124892F0895882339F04298000096
:10059000419A0000429A0000089542980000419854
:1005A0000000429A00000895429A000086B14298E5
:1005B0000000817008950F931F93082F5C9A429852
:1005C0005C9810E0802F80780E94C402000F1F5FAB
:1005D0001830C1F742981F910F9108958F770E94AC
:1005E000DB0208950F931F93082F10E0802F80786F
:1005F0000E94C402000F1F5F1830C1F742981F917C
:100600000F9108950F931F93429880E000E0182FF8
:10061000110F0E94D402810F0F5F0830C1F71F91A4
:100620000F9108950E94EE020E9402035C9A0895C1
:100630001F93162F80680E94DB02812F0E94F20216
:100640005C9A1F9108951F931091F9021827E0EF0B
:10065000F2E0E80FF11D89E767850E9418038DE33A
:10066000612F0E94180382E4612F0E9418031F91DA
:10067000089586E20E94120308950F931F938BE260
:100680000E941203082F8CE20E941203282F30E0F0
:1006900016E0369527951A95E1F710E0000F111F27
:1006A000000F111F202B312BC9011F910F910895AD
:1006B0000F931F938C018CE1F80164810E94180351
:1006C0008DE1F80165810E9418038EE1F8016681D1
:1006D0000E94180380E2F80167810E94180381E2FA
:1006E000F80160850E94180382E2F80161850E948A
:1006F000180383E2F80162850E94180384E2F8017E
:1007000063850E94180385E2F80164850E9418033E
:100710008AE2F80165850E9418038EE6F801668575
:100720000E9418038FE6F80167850E94180380E78E
:10073000F80160890E94180381E7F80161890E942D
:10074000180382E7F80162890E9418031F910F9134
:100750000895EF92FF920F931F93CF93DF937B0146
:100760008C01603028E372072CE982072CE19207A4
:1007700028F520E836E948E950E00E94E820E90140
:100780006897B90180E090E020E839E647E65FEF3E
:100790000E94B5206E0D7F1D801F911F22E0660F05
:1007A000771F881F991F2A95D1F721E732E040E093
:1007B00050E00E94E820890180E421C020E03DE271
:1007C00041E351E00E94E820E9016897B90180E027
:1007D00090E020E033ED4EEC5EEF0E94B5206E0D10
:1007E0007F1D801F911F660F771F881F991F21E7AC
:1007F00032E040E050E00E94E820890180E69E015E
:100800002F71622F680F85E70E94180386E7612F1A
:100810000E94180387E7602F0E941803CDB7DEB748
:10082000E6E00C944D219F92AF92BF92CF92DF925F
:100830000F93DF93CF9300D000D0CDB7DEB7982EC3
:1008400083E00E9412038093190384E00E94120344
:1008500080931A0386E060E00E94180387E061E05D
:100860000E94180389E06FE70E9418038AE065E0A0
:100870000E9418038BE062E10E9418038CE065E19E
:100880000E9418038DE06DEF0E9418038EE060E077
:100890000E941803992019F08FE492E008C080911B
:1008A000170323E1829FC001112480519E4F0E94B3
:1008B000580380E36CE80E94180382E36FE00E9413
:1008C000180383E362E40E94180384E36AE00E9451
:1008D000180385E36AE20E94180386E36DE20E9432
:1008E000180387E364ED0E94180388E360E00E9428
:1008F000180389E360E00E941803992049F055E845
:10090000A52E51ECB52E51ECC52E5EEDD52E08C0AE
:10091000A090F902B090FA02C090FB02D090FC02C5
:100920000AE38D2D9927AA27BB2789839A83AB8356
:10093000BC83802F69810E941803802F8B5F69819F
:100940000E941803DC2CCB2CBA2CAA240F5F0E3388
:1009500041F783E46FEF0E94180384E46FEF0E9475
:10096000180385E46FEF0E94180386E46FEF0E947E
:100970001803992019F08DE666E003C08DE66091BA
:10098000FD020E94180389E760E00E9418038AE7CD
:100990006091FE020E94180383E760E00E94180342
:1009A00084E760E00E941803992029F060EC72E966
:1009B0008DEE99E108C06091F5027091F602809188
:1009C000F7029091F8020E94A9030F900F900F90E8
:1009D0000F90CF91DF910F91DF90CF90BF90AF90AC
:1009E0009F90089587E061E00E9418038EE764E21B
:1009F0000E94180388E063E00E94180388E060E02A
:100A00000E94180387E065E00E94180385E062E019
:100A10000E94180383E00E9412038093190384E06C
:100A20000E94120380931A03089590E0411191E00F
:100A3000880F982B9093BA00660F6093BD00309397
:100A4000200320931F030895882311F085EC01C033
:100A500085E88093BC00089585ED8093BC0080916B
:100A6000BC0084FDFCCF089585EC8093BC00089504
:100A7000ECEBF0E0108285E480831092250308956A
:100A80001F920F920FB60F9211242F933F934F9303
:100A90005F936F937F938F939F93AF93BF93EF93E6
:100AA000FF93DF93CF930F92CDB7DEB78091B9005C
:100AB00090E0887F90708036910509F4EAC0813615
:100AC0009105CCF58832910509F47CC089329105F5
:100AD000B4F48031910509F470C0813191053CF482
:100AE000009709F40EC1089709F00DC166C088315E
:100AF000910509F467C0809709F005C177C080347B
:100B0000910509F490C08134910544F48033910536
:100B100009F46EC0C89709F0F6C06CC08035910525
:100B200009F471C08835910509F483C088349105B2
:100B300009F0E9C0A5C08839910509F4DCC08939FC
:100B40009105ECF48837910509F4A3C08937910524
:100B50004CF48836910509F49CC08037910509F062
:100B6000D2C097C08838910509F4C5C08039910575
:100B700009F492C08038910509F0C5C08DC0803B52
:100B8000910509F4A5C0813B91054CF4803A91058B
:100B900009F499C0883A910509F0B5C099C0803C24
:100BA000910509F4AAC0883C910509F4A6C0883BC8
:100BB000910509F0A8C080E08CC08091210380934A
:100BC000BB009BC0809124038150809324038F5FDE
:100BD00009F43FC0E0912203F091230381918093B7
:100BE000BB00F0932303E093220387C082E049C057
:100BF00083E047C084E080932603809125038B7FA8
:100C00008093250362C08091BB00E0912203F091A4
:100C100023038193F0932303E09322038091240321
:100C200081508093240380912403823008F065C0B2
:100C300062C08091BB00E0912203F0912303819375
:100C4000F0932303E0932203809124038150809347
:100C50002403809125038B7F8093250380912503B6
:100C600080FF4FC0809125038E7F80932503809164
:100C7000250382608093250384EA8093BC0043C0EF
:100C800085E080932603809125038B7F8093250345
:100C900038C01092240331C0E0911F03F09120036B
:100CA000309749F19091BB00809124038F5F80932E
:100CB0002403815011F060E001C062E09983CE010D
:100CC000019609951BC00E942C050E9434051BC08B
:100CD00081E0E0911F03F0912003309761F08823B9
:100CE00011F461E001C063E0CE010196099599819C
:100CF0009093BB0003C080E001C081E00E94240506
:100D000002C00E942C050F90CF91DF91FF91EF91CF
:100D1000BF91AF919F918F917F916F915F914F9113
:100D20003F912F910F900FBE0F901F90189525B1F6
:100D300090E0FC01EE0FFF1FE80FF91FE457FC4F96
:100D40008081282B25B988B19181892B88B98BB1F5
:100D50009281892B8BB9089585B19091BC03892329
:100D600085B988B19091BD03892388B98BB19091E1
:100D7000BE0389238BB908951F920F920FB60F926D
:100D800011241F932F933F934F935F936F937F9300
:100D90008F939F93AF93BF93CF93DF93EF93FF9383
:100DA00010915F0380918602C0918402D0918502E8
:100DB000181708F05BC08091BF039091C003909317
:100DC000870080938600E12FF0E0EE0FFF1FEE59C1
:100DD000FD4F808191810E947702880F991F909327
:100DE000C0038093BF038091BF039091C0039E0115
:100DF000281B390BC901309385022093840220916E
:100E0000EB023091EC02220F331F8217930720F47C
:100E1000309385022093840280916103882339F402
:100E20008091E30280FF59C0183008F456C08FEF5C
:100E30009FEF909389008093880080918400909127
:100E400085008097D0F30E94AC06809160038823D0
:100E500039F480915F03882319F081500E9497062E
:100E600080915F038F5F80935F033EC08091BF03DB
:100E70009091C0039093870080938600D093C00325
:100E8000C093BF0380916103882319F08FEF9FEF18
:100E900006C08091BF039091C00388559240909303
:100EA00089008093880080E49CE990938502809378
:100EB000840280918400909185008097D0F30E94F5
:100EC000AC0680916003882329F4809186028150CA
:100ED0000E94970610925F0307C08091BF03909114
:100EE000C00388559240A5CFFF91EF91DF91CF913C
:100EF000BF91AF919F918F917F916F915F914F9132
:100F00003F912F911F910F900FBE0F901F9018953A
:100F100090E0880F991F880F991F8C30910518F465
:100F20002CE030E007C09C0183E0253F380710F03B
:100F300024EF33E0C90108950F931F930091E40259
:100F40000033C0F4202F30E0C90180739070009707
:100F500019F0409749F403C08091590307C080916C
:100F60005E038295807F02C08091580389010F70D3
:100F7000107016C00F33E8F410E00F7010708091FD
:100F80005E038295807F0E948807F801EE0FFF1FA5
:100F9000EE59FD4F918380830F5F1F4F809158035F
:100FA0000E948807000F111F0E591D4FF8019183F1
:100FB00080831F910F9108951F93809163039091F7
:100FC00064038F5F9F4F39F11091E402412F50E08D
:100FD0004F705070BA016F5F7F4FA3E6B3E020E01F
:100FE00030E02417350789F02617370711F410333E
:100FF00060F4F8948D919C911197F901EE0FFF1F09
:10100000EE59FD4F9183808378942F5F3F4F129666
:101010002031310531F71F9108951F93CF93DF934E
:10102000EC0170E0CB018270907060FF1AC0892BD8
:1010300031F08091850388831092030445C010919C
:10104000030480EF92E00E941E011817D8F5E12FEB
:10105000F0E0EF53FC4F808188831F5F10930304FF
:1010600033C0892BC1F0988190930204109203043D
:10107000892F807E803651F480918503823010F173
:1010800088818F718093430383E01AC09E3FE1F40F
:101090001092850317C0809102048F3FA9F420911C
:1010A0000304293278F4E22FF0E0E051FD4F88810B
:1010B0008083822F8F5F80930304893229F481E03B
:1010C0008093850380E001C081E0DF91CF911F9183
:1010D0000895EF92FF920F931F93CF93DF9380E2D7
:1010E00060E040E02DE038E00E9415051092850395
:1010F00092E0E92E85E0F82E04E0809185038130AE
:1011000039F480E00E941304E09285034398F5CF00
:1011100010918503133061F42D98809143030E9450
:1011200023031093D4020E94F20400938503E5CFB9
:1011300080918503843009F78091D4028430E9F6E8
:101140008FE70E94EE02C0E0D0E007C00E940203D9
:10115000FE01EF53FC4F8083219680EF92E00E94C6
:101160001E0190E0C817D9078CF3F09285032D9AE1
:10117000C4CFA0E0B0E0EFEBF8E00C942D21EC013F
:101180000E94811B5B016C017E0100E010E011C038
:10119000209779F00E94811B6A197B098C099D09AF
:1011A000E616F7060807190720F40E94380581E0C3
:1011B00008C08091250382FDEBCF80912603109219
:1011C0002603CDB7DEB7EAE00C944921A0E0B0E0F9
:1011D000ECEEF8E00C942F21182F7B01042FC22F86
:1011E000D0E024E0C22ED12CCC22DD22C2FF03C0ED
:1011F00080E090E004C080918202909183020E947E
:10120000B908282F8823B9F51092260300932403E8
:10121000F0922303E0922203110F11601093210337
:1012200090912503C1FD02C084E001C085E0892BB7
:10123000809325038091250381FF0BC080912503B6
:101240008D7F80932503809121038093BB0085ECE3
:1012500001C085EE8093BC00C0FF0DC0C114D10455
:1012600019F080E090E004C08091820290918302A6
:101270000E94B908282F822FCDB7DEB7E8E00C9482
:101280004B21A0E0B0E0E7E4F9E00C942F21182F07
:101290007B01042FC22FD0E034E0C32ED12CCC220E
:1012A000DD2222FF03C080E090E004C08091820232
:1012B000909183020E94B908282F8823B1F51092DB
:1012C000260300932403F0922303E0922203110FDC
:1012D0001093210390912503C1FD02C084E001C059
:1012E00085E0892B809325038091250381FF0BC026
:1012F000809125038D7F8093250380912103809326
:10130000BB0085EC01C085EE8093BC00C0FF0DC022
:10131000C114D10419F080E090E004C080918202F1
:10132000909183020E94B908282F822FCDB7DEB793
:10133000E8E00C944B218091D402813011F081E0DF
:1013400008950E94811B20911B0330911C03409142
:101350001D0350911E03621B730B840B950B615A86
:1013600076488140904010F480E0089582E008952E
:10137000FF920F931F93CF93DF93182F092FF62E11
:101380008EE30E941803212F302FC901EC0110E0D9
:1013900005C08FE769910E9418031F5F1F15C8F3EE
:1013A00085E064E00E94180383E00E9412038093AA
:1013B000190384E00E94120380931A030E94811B88
:1013C00060931B0370931C0380931D0390931E0373
:1013D00087E069E00E94180381E08093D402CDB7D2
:1013E000DEB7E5E00C944E210E94B8098091D4024A
:1013F0008130D9F40E94811B20911B0330911C0382
:1014000040911D0350911E03621B730B840B950BBF
:10141000605A76488140904040F4E8CF8CE994E0EF
:1014200060E071E00E94691E08958091D4028130CD
:10143000A9F30895A1E0B0E0E0E2FAE00C943521D0
:10144000809185038230B9F480E2BE016F5F7F4FE7
:1014500041E021E00E94E608882379F08FEF809335
:1014600085030E94731B60938603709387038093A8
:101470008803909389038FEF01C089812196E2E070
:101480000C945121A1E0B0E0E8E4FAE00C9435219D
:10149000809185038230D9F480914303805A8983F7
:1014A00080E2BE016F5F7F4F41E021E00E94410971
:1014B000882369F08FEF809385030E94731B6093EC
:1014C0008603709387038093880390938903219602
:1014D000E2E00C945121AAE2B0E0E1E7FAE00C94DA
:1014E00033218FEF8983DE011296E0EFF2E089E28B
:1014F00001900D928150E1F780E28E010F5F1F4F46
:10150000B8014AE221E00E944109882351F480E2B7
:10151000B80141E021E00E94E608882311F482E04E
:1015200001C08FEF8093850380918503823051F055
:101530000E94731B609386037093870380938803D4
:1015400090938903AA96E4E00C944F21A2E0B0E0C6
:10155000ECEAFAE00C9431210E94811B9B01AC0162
:101560008091270390912803A0912903B0912A0329
:1015700079018A01E81AF90A0A0B1B0BD801C70185
:1015800081519742A040B04008F444C080912B03A1
:101590008F5F80932B03815080FD02C000E001C06B
:1015A00007E02093270330932803409329035093A7
:1015B0002A038CE994E063E00E9421208CE994E006
:1015C00061E00E94212077E0F72EF00E802F90E05E
:1015D000880F991F9C012E593D4F3A832983F901A9
:1015E00060817181672F772763707070880F991FF2
:1015F000682B792B8CE994E00E942120E981FA8103
:101600006081718170708CE994E00E9421200F5FED
:101610000F15E1F62296E6E00C944D211F93182F4A
:101620008CE994E0612F0E942120812F0E94C80044
:101630001F910895A0E0B0E0E0E2FBE00C942F21C0
:10164000082F0E94811B9B01AC0180912703909180
:101650002803A0912903B0912A0369017A01C81ACD
:10166000D90AEA0AFB0AD701C60181519742A04074
:10167000B04008F443C020932703309328034093DD
:10168000290350932A03109206041092050488EA55
:101690000E940E0B002311F481E001C081E80E943A
:1016A0000E0B80E10E940E0BC0E0D0E0FE01EE0FB9
:1016B000FF1FEE59FD4F808191810E9477028C01BE
:1016C000E3E0000F111FEA95E1F7812F0E940E0B56
:1016D000802F0E940E0B2196C031D10539F7609101
:1016E00006048CE994E00E94212060910504709129
:1016F000060470708CE994E00E942120CDB7DEB71B
:10170000E8E00C944B21A0E0B0E0E9E8FBE00C94A9
:101710002F21182F062F0E94811B9B01AC01809165
:10172000270390912803A0912903B0912A0369010E
:101730007A01C81AD90AEA0AFB0AD701C6018151FF
:101740009742A040B04008F4D6C1209327033093BD
:1017500028034093290350932A03809162029091B9
:101760006302880F991F80932C03977080912D033B
:10177000887F892B80932D0320916402309165022C
:10178000220F331F922F990F990F990F8770892B72
:1017900080932D03422F42954695477080912E03EA
:1017A000807C932F9770990F990F990F842B892B19
:1017B00080932E032091660230916702220F331F1F
:1017C000922F9295990F990F907C8F73892B80930C
:1017D0002E03932F9295990F990F907C822F8695C7
:1017E0008695892B80932F03932F969596959170CC
:1017F000809130038E7F892B809330032091680283
:1018000030916902220F331F922F990F8170892B1B
:1018100080933003422F441F4427441F809131039B
:10182000807F932F9770990F842B892B809331039E
:1018300020916A0230916B02220F331F922F9295F2
:10184000907F8F70892B80933103422F42954F7088
:10185000809132038078932F97709295907F842B9C
:10186000892B8093320320916C0230916D02220FFC
:10187000331F8F7780933203932F979599279795EE
:10188000822F8695892B80933303932F969593709F
:10189000809134038C7F892B8093340340916E02B6
:1018A00050916F02440F551F942F990F990F837019
:1018B000892B80933403942F9295969596959370E7
:1018C00020913503207E852F8770880F880F292B64
:1018D000282B209335038091700290917102880F1C
:1018E000991F382F3295330F307E2F71232B209381
:1018F0003503292F2295220F207E86958695869581
:10190000822B809336038091720290917302880F2C
:10191000991F80933703977080913803887F892BB4
:10192000809338032091740230917502220F331F87
:10193000922F990F990F990F8770892B80933803F5
:10194000422F42954695477080913903807C932FB2
:101950009770990F990F990F842B892B80933903D6
:101960002091760230917702220F331F922F9295A9
:10197000990F990F907C8F73892B80933903932F44
:101980009295990F990F907C822F86958695892B39
:1019900080933A03932F96959695917080913B038F
:1019A0008E7F892B80933B032091780230917902BE
:1019B000220F331F922F990F8170892B80933B0345
:1019C000422F441F4427441F80913C03807F932F64
:1019D0009770990F842B892B80933C0320917A0276
:1019E00030917B02220F331F922F9295907F8F7040
:1019F000892B80933C03422F42954F7080913D0389
:101A00008078932F97709295907F842B892B809369
:101A10003D0320917C0230917D02220F331F8F778E
:101A200080933D03932F979599279795822F8695BD
:101A3000892B80933E03932F9695937080913F035B
:101A40008C7F892B80933F0340917E0250917F02CF
:101A5000440F551F942F990F990F8370892B8093F2
:101A60003F03942F929596959695937020914003FD
:101A7000207E852F8770880F880F292B282B209395
:101A800040038091800290918102880F991F382F26
:101A90003295330F307E2F71232B20934003292F53
:101AA0002295220F207E869586958695822B80939F
:101AB0004103112311F490E001C098E0002311F4D8
:101AC00080E001C084E0892B809342038CE994E09C
:101AD0006FE00E942120CCE2D3E08CE994E0699190
:101AE0000E94212083E0C334D807B9F78CE994E041
:101AF00060E00E942120CDB7DEB7E8E00C944B21D6
:101B00001F93182F8091DE028B3221F48CE0612F1D
:101B10000E947C1C8091D602873259F4112321F057
:101B20008091B000806103C08091B0008F7E80936F
:101B3000B0001F91089580915C0390915D039F77A1
:101B40000E949C02982F80935E038F3029F480912D
:101B500058038695805804C089E0989FC0011124DD
:101B600080935903F8940E949C0778948091D60240
:101B70008132C9F490915903892F81508E3F60F0D2
:101B80008091B0008F7D8093B00060E0911161E0A2
:101B900083E00E947C1C08959093B4008091B00073
:101BA00080628093B00008951F93182F811111E077
:101BB00082E1612F0E947C1C83E1612F0E947C1CCA
:101BC00010922403109225038091B9008C6F8093AA
:101BD000B90080E28093B80085E48093BC001F9137
:101BE0000895CF93DF938CE994E00E94AE1F892B78
:101BF000F9F080910004C82FD0E09E012F5F3F4F85
:101C00002F7130708091FF0390E02817390781F021
:101C10008CE994E00E94E81FC152DC4F88838091D8
:101C2000000490E001968F71907080930004DBCFE8
:101C3000DF91CF910895EF92FF921F93CF93DF939F
:101C400080EF92E00E942801482F809386025091F5
:101C5000E402252F30E02F70307090E0281739070C
:101C600019F44F5F4093860250535F3058F440910F
:101C70008602842F90E001972817390719F44F5FE7
:101C80004093860280918602813118F080E1809332
:101C90008602ECE8F3E0108211821282339623E090
:101CA000E33BF207C1F78FEF8093BC038093BD0342
:101CB0008093BE0386EDE82E82E0F82EA5E9B2E01F
:101CC000E7016FEF5FEF4FEF88818031F0F490E034
:101CD0003C91FC01EE0FFF1FE80FF91FE457FC4F8A
:101CE0008081832B808311962C9111978181822B87
:101CF000818312969C9112978281892B82833095E1
:101D0000432320955223909569232196139682E0D0
:101D1000C33ED807C9F66093BE035093BD034093FA
:101D2000BC03C8E8D2E010E0F7018081823238F0CD
:101D30008632B0F0863219F4888160E00FC01B3023
:101D400021F48091C1008F7E05C01C3029F4809160
:101D5000C100877F8093C100888161E00E94101CD0
:101D60001F5F0894E11CF11C21961D30E9F680915B
:101D7000DB02803231F489E061E00E947C1C82E861
:101D800001C082E08093800081E0809360038093B3
:101D900061038091D602813211F08732D9F483E059
:101DA00061E00E94101C83E060E00E947C1C809136
:101DB000D602813231F481E08093B0008093B1008B
:101DC00009C082E08093B00085E08093B1008EE38B
:101DD0008093B3008AE1809381008FEF9FEF90930F
:101DE00089008093880080ED97E09093870080932E
:101DF000860080E49CE9909385028093840290930E
:101E0000C0038093BF0310925F0380916F008160D5
:101E100080936F008091E30283FF0DC08091630384
:101E2000909164038F5F9F4F31F00E94DC07109206
:101E3000610310926003DF91CF911F91FF90EF90AB
:101E400008958EE060E00E94101C8FE061E00E9427
:101E5000101C80E161E00E94101C82E060E00E94A2
:101E6000101C84E061E00E94101C089583E00E9431
:101E700012038093190384E00E94120380931A03D3
:101E800087E061E00E9418036AE070E080E090E083
:101E90000E94A71B0E94F204000008950F931F9355
:101EA000082F17C0439A64E670E080E090E00E943B
:101EB000A71B439864E670E080E090E00E94A71BB7
:101EC0001F5F101778F36CE271E080E090E00E94F1
:101ED000A71B10E0F6CF482F392F25E00DC0F99948
:101EE000FECF1FBA842F932F92BD81BD60BD0FB668
:101EF000F894FA9AF99A0FBE215059F0F999FECF49
:101F0000842F932F92BD81BDF89A80B5681739F759
:101F1000089582E00E944E0F0895A0E0B0E0E3E94A
:101F2000FFE00C942721482E562EEE24FF24C0E01B
:101F3000D0E0CC24DD248824992404C05524539473
:101F4000CC24DD24442051F465EDE62E62E0F62E2B
:101F5000C0E0D0E05BE1852E912C19C021E0421653
:101F600051F440EFE42E42E0F42ECDE1D0E039E22E
:101F7000832E912C0CC032E0431649F423E6E22E66
:101F800023E0F22EC8E4D0E090E2892E912C3E01AD
:101F90006C0C7D1C1092060410920504E3011BC01A
:101FA000552059F4F999FECFD2BDC1BDF89A80B53C
:101FB000F701E00FF11F808307C0F701E00FF11F69
:101FC000CE0160810E946B0F0E0D1F1DF8018081F4
:101FD0000E94C80021969E012619022F10E00815C4
:101FE0001905F0F2CE015520D9F4F999FECFD2BDF2
:101FF000C1BDF89A20B5F999FECF2196D2BDC1BDD9
:102000002197F89A80B590E0B22EAA248A299B29BC
:1020100020910504309106042817390759F48ECF12
:102020002196609106040E946B0FCE016091050419
:102030000E946B0F80E091E0C80ED91E91E0C91696
:1020400093E0D90608F47ECF852DCDB7DEB7E0E169
:102050000C94432182E060E00E948D0F882331F4CC
:102060008FEF9FEF9093640380936303089582E062
:1020700061E00E948D0F0895282F81E08093D502A2
:1020800081E28093D602E7EDF2E080E081938F5FFA
:102090008830E1F786E28093DF028093E00284E2F9
:1020A0008093E10285E28093E20282E08093E30282
:1020B0008FEF8093E4029AE09093ED021092EE028B
:1020C0001092EF021092E5021092E6021092E702DF
:1020D0001092E8028EE18093E9029093EA0288EB85
:1020E0009BE09093EC028093EB02222361F080E06E
:1020F00061E00E948D0F8FEF9FEF909364038093B8
:1021000063030E9437100895ADE5B0E0EAE8F0E11E
:102110000C9425215B016C010E94731B1B012C0197
:1021200081E00E94130483E08093D4020E94360F62
:102130008CE994E06CE071E00E94691E3E01089415
:10214000611C711CE3C08CE994E06AE171E00E94BB
:10215000691E8FE70E94EE020E940203182F8983F6
:10216000823601F500EF12E00E940203F80181932C
:102170008F01F3E009311F07B9F78091F00287332F
:1021800009F0BFC08CE994E063E271E00E94691E2F
:1021900082E48983CE01019661E00E94F4092D9AC0
:1021A00081E0CAC0803719F0893631F506C020E5D4
:1021B0002A83AA24BB24650105C081E00E943C104B
:1021C00089E48A8380910404882321F08091E302CA
:1021D000806803C08091E3028F778093E302DE0181
:1021E0001396E5EDF2E08BE101900D928150E1F75D
:1021F000CE0102966CE183C08437D9F434E53E8F7A
:1022000083E08F8F93E798A3EDE0E9A3EAA3DE01D3
:102210009396E6EDF1E08AE101900D928150E1F7AD
:10222000CE014E966FE10E94F409AA24BB246501F9
:1022300068C0853791F405ED12E00E940203F801B1
:1022400081938F01F2E0003F1F07B9F780E061E062
:102250000E948D0F25E5298350C0863631F5809187
:102260006303909164038F5F9F4FD1F086E48DAF3D
:1022700073E6E72E73E0F72E8E01025C1F4FF70125
:10228000819191917F010E947702F801908381836F
:102290000E5F1F4FF3E8EF16F3E0FF0681F701C072
:1022A0001DAFCE01CD9661E22AC08736D9F403E690
:1022B00013E00E940203982E88240E9402039401D6
:1022C000280F311DC9010E944802F80181939193A2
:1022D0008F01F3E003381F0761F727E429830E9489
:1022E00037100BC0873469F48FEF9FEF909364032E
:1022F000809363030E9437101983C30161E00E9439
:10230000F40993E09093D4020E94F204A114B10462
:10231000C104D10459F00E94731B62197309840926
:1023200095096A157B058C059D0528F48091D402DA
:10233000843061F708CF80E0C35ADF4FE2E10C94AC
:10234000412180E060E00E948D0F882319F481E034
:102350000E943C10089581E061E00E948D0F089575
:1023600081E060E00E948D0F882311F490E006C0A8
:1023700090E08091F002873309F491E0892F08956D
:10238000EF92FF920F931F93CF93DF93EB019C018A
:10239000442737FD4095542F60E271EA87E090E0D2
:1023A0000E940A2189011216130614F001E010E0C0
:1023B000BE01882777FD8095982F20E231EA47E01B
:1023C00050E00E94B5209801442737FD4095542FD6
:1023D0000E940A217901C0E0D0E009C0419AC801F9
:1023E0000E94CB1B4198C8010E94CB1B2196CE15A1
:1023F000DF05A4F3CDB7DEB7E6E00C944D211F93C3
:10240000182F2D9A83E00E9412038093190384E011
:102410000E94120380931A0386E060E00E94180372
:1024200087E061E00E94180389E06FE70E941803CB
:102430008AE065E00E9418038BE062E10E941803C5
:102440008CE065E10E9418038DE06DEF0E94180397
:102450008EE060E00E94180380E76CE20E9418039F
:1024600080E360E00E94180389E760E00E9418039F
:102470008AE765E00E94180381E762E10E94180381
:1024800082E762E00E94180383E760E00E9418037D
:1024900084E760E00E9418036091E5027091E60213
:1024A0008091E7029091E8020E94A9038DE667E01F
:1024B0000E9418036AE070E080E090E00E94A71B91
:1024C00087E069E00E9418036AE070E080E090E035
:1024D0000E94A71B112369F010E007C088EB91E070
:1024E00061E070E00E94C011A8951F5F1531B1F73F
:1024F0004BC088E891E061E070E00E94C011A895AF
:102500008DE665E00E9418036AE070E080E090E0EC
:102510000E94A71B88EB91E061E070E00E94C0116F
:10252000A8958DE664E00E9418036AE070E080E000
:1025300090E00E94A71B8DE591E061E070E00E94B1
:10254000C011A8958DE662E00E9418036AE070E071
:1025500080E090E00E94A71B8FEA90E061E070E0CD
:102560000E94C011A8958DE660E00E9418036AE001
:1025700070E080E090E00E94A71B85E091E062E0BF
:1025800070E00E94C011A89587E061E00E941803E6
:102590002D981F910895A6E1B0E0E1EDF2E10C94D1
:1025A0002721A8958CE00E941203882359F48CE916
:1025B00094E06EE271E00E94691E80E00E941304C4
:1025C0000E94360F0E94F10D0E94811B0E941A0A80
:1025D00090E0853009F491E08E010F5F1F4FBB241E
:1025E000BA948091D402843019F0992309F488C1F7
:1025F0000E94811B6B017C018091D4028430F1F434
:102600008FE70E94EE0200E010E008C00E94020383
:10261000F801EF53FC4F80830F5F1F4F80EF92E074
:102620000E941E0190E00817190784F30E943D03E1
:1026300090935B0380935A032D9A29C080EF92E018
:102640000E941E01482F4F5F80E2B80121E00E94E6
:10265000E608882371F0B09285030E94731B609393
:10266000860370938703809388039093890390E097
:10267000B8CF80EF92E00E941E01482F21EC33E09A
:10268000FE013296C901BF0150E00E948C00C09249
:102690004403D0924503E0924603F0924703109220
:1026A000840380915C0390915D03880F991F816082
:1026B00090935D0380935C03439880E00E94800DBB
:1026C0008091C103282F30E0C9018E739070892B4F
:1026D00099F5F89480911803877062E672E042ECF5
:1026E00053E00E94AC010E949C0778948091C10342
:1026F00090918B0380FF1BC0992309F045C0A3E68E
:10270000B3E020E030E0F901EE0FFF1FEE59FD4F7E
:10271000808191818D939D932F5F3F4F20313105B3
:1027200091F70E94371081E080938B032DC099238D
:1027300059F110928B0328C0C90188739070C89713
:1027400019F54091D603842F822787FF1DC040587A
:102750004093D6038091E2028532B1F410E00AC0C2
:102760001F5FE12FF0E0EF53FC4F8CE994E06081B4
:102770000E942120212F30E08091C10390E08770DA
:1027800090708217930764F780918303882319F46C
:1027900081E0809383031092620310926003109291
:1027A000610380911803887109F4A1C04091D60398
:1027B0008091C10390E0242F30E08227932786FD8B
:1027C00060C0407C80E448274093D6039091FF038B
:1027D00080910004981701F1A7EDB3E030E00FC03D
:1027E0003F5F892F90E0FC01E152FC4F20812D9347
:1027F00001968F7190708093FF03383031F0909183
:10280000FF0380910004981759F7395C8091D60333
:10281000382B3093D60335C0809157038093D7036C
:102820008091DF02863251F482E10E94DF1C95958F
:102830008795959587958093D80302C01092D80309
:102840008091E002863251F483E10E94DF1C95956D
:102850008795959587958093D90302C01092D903E7
:1028600080915B038093DA0380915A038093DB03AA
:1028700080915C0390915D039F770E949C028093FE
:10288000DC0386ED93E069E00E94B80902C00E9473
:10289000F10D0E949B098823D1F306ED12E088E830
:1028A000E82E82E0F82EF8018081E82FF0E0CF01D9
:1028B000807F9070409791F4EF70F070EE0FFF1FE3
:1028C000EE59FD4F8081918160E08F3F910511F0BD
:1028D00008F061E0F70180810E947C1C0F5F1F4FB0
:1028E0000894E11CF11CF2E0033E1F07E1F683E0CF
:1028F0008093D4020E94F20481E080938A032D9891
:102900000E94811B5B016C010E94731B2B013C0127
:1029100080918403823008F065C0E0904403F09019
:10292000450300914603109147038091480390911D
:102930004903A0914A03B0914B038E159F05A00750
:10294000B10709F44FC080EF92E00E943801A60160
:1029500095012E193F09400B510B6C5D754080406D
:1029600090406217730784079507E0F5E0924803EB
:10297000F092490300934A0310934B030E943903DA
:10298000809357032091550330915603280F311D32
:102990003093560320935503609154036F5F609307
:1029A00054036930F8F0C90170E00E94D420CB01D3
:1029B00070935603609355032091580343E0249F7E
:1029C00090011124820F931F969587959695879570
:1029D000809358030E949B0D10925603109255034A
:1029E000109254038091830390900104882309F48A
:1029F00063C180908403891408F0E1C180EF92E004
:102A00000E943801209144033091450340914603D0
:102A100050914703A21AB30AC40AD50A68517C4FE1
:102A20008F4F9F4F6A157B058C059D0508F077C079
:102A300080915C0390915D03880F991F90935D03D3
:102A400080935C0381E080938A03882081F4409224
:102A50004C0350924D0360924E0370924F031092BC
:102A6000500310925103109252031092530380911D
:102A700084038F5F8093840380EF92E00E9438018B
:102A80002091440330914503409146035091470300
:102A9000260F371F481F591F2093440330934503C7
:102AA000409346035093470381E080938A03439AFF
:102AB0000E94800D0E949B0D32C080EF92E00E9428
:102AC00038019B01AC018091440390914503A09192
:102AD0004603B091470386017501E81AF90A0A0B0B
:102AE0001B0B682D70E080E090E00E94B5206E1511
:102AF0007F058007910798F410925D0310925C03A4
:102B000081E080938A03109258030E949B0DA0924B
:102B10004403B0924503C0924603D092470380918C
:102B20008403882309F4F2C09091ED02992389F17E
:102B300080916203882369F5892F90E00E94E50067
:102B400020914C0330914D0340914E0350914F031F
:102B500083017201E21AF30A040B150B6E157F054F
:102B600080079107B0F481E0809362030E94DC0744
:102B70008091E9020E941801640D751D861D971D44
:102B8000616060935003709351038093520390935C
:102B900053039091EF029923F1F080916003882311
:102BA000D1F4892F90E00E94E50020914C033091F0
:102BB0004D0340914E0350914F0383017201E21A7D
:102BC000F30A040B150B6E157F058007910718F4A7
:102BD00081E0809360039091EE029923F1F080915F
:102BE00061038823D1F4892F90E00E94E5002091B1
:102BF0004C0330914D0340914E0350914F0383019C
:102C00007201E21AF30A040B150B6E157F0580079B
:102C1000910718F481E0809361038091E50290911F
:102C2000E602A091E702B091E8020097A105B10584
:102C300009F46CC08091500390915103A09152030C
:102C4000B09153030097A105B10509F45FC083015A
:102C50007201E81AF90A0A0B1B0B17FD57C06091A5
:102C6000EA0270E080E090E028EE33E040E050E0DF
:102C70000E94B5206E157F058007910708F046C0B9
:102C80008091E30290E0E4E096958795EA95E1F77C
:102C900081700E94FF1180E00E9413040E94F204E0
:102CA0000E94731B61606093500370935103809383
:102CB0005203909353032AC080EF92E00E943801A0
:102CC0009B01AC018091440390914503A091460380
:102CD000B091470386017501E81AF90A0A0B1B0B2C
:102CE000692D70E080E090E00E94B5206E157F05B0
:102CF0008007910758F4A0924403B0924503C09214
:102D00004603D092470381E080938A038091610358
:102D10008823B1F48091E202883219F40E94A60A55
:102D20000FC0893239F480916203609184030E945C
:102D3000830B06C08A3221F4809162030E941A0B31
:102D400080918A038823B9F0E0914303EF5FE09319
:102D50004303E83131F0F0E0E051FD4F87858823EF
:102D600011F410924303809143030E9423030E94B5
:102D7000420A10928A03809185038F3F21F50E94B9
:102D8000731B2091860330918703409188035091F3
:102D90008903621B730B840B950B695E7340804043
:102DA000904088F00E94731B6093860370938703A2
:102DB00080938803909389030E946B0A04C089144E
:102DC00009F0ADCE7ACE6696E0E10C944321FF92F5
:102DD0000F931F93082FF62E61E00E94101C802F86
:102DE00061E00E947C1C8F2D61E00E947C1C8AE0C7
:102DF00090E00E94CB1B8F2D0E94AF1C892B11F4F9
:102E000010E00FC0802F60E00E947C1C8AE090E000
:102E10000E94CB1B8F2D0E94AF1C10E0892B09F460
:102E200011E0802F60E00E94101C802F60E00E9463
:102E30007C1C8F2D60E00E947C1C812F1F910F91C4
:102E4000FF900895EF92FF920F931F937C010CE97E
:102E500014E0C8016F2D70E04AE050E00E94E61DCA
:102E6000C8016EE20E94251DB701E4E076956795E2
:102E7000EA95E1F76F707070C8014AE050E00E9477
:102E8000E61DC8016EE20E94251D8FE0E822FF24A6
:102E9000C801B7014AE050E00E94E61D1F910F9162
:102EA000FF90EF900895A2E2B0E0E9E5F7E10C941D
:102EB00025218E010F5F1F4F80E1D8011D928A9559
:102EC000E9F78CE994E066E371E00E94691E0E94D4
:102ED000360F20E431EE4DE958E12F8F38A349A396
:102EE0005AA380EC91EDA8E9BBE18B8F9C8FAD8F4D
:102EF000BE8F24EF31E040E050E02F8B388F498FB8
:102F00005A8F80E5C82E83ECD82EE12CF12CB0E44A
:102F10004B2EB1EE5B2EBDE96B2EB8E17B2E8824E3
:102F20009924540133241E8A1D8A198A1A8A1B8AFD
:102F30001C8AFFC08CE994E00E94E81F8434B9F039
:102F4000853430F48332B9F18C3209F0CCC044C0FE
:102F5000833509F0C8C02F8D38A149A15AA1C901F4
:102F6000DA012C013D01882499245401E2C08CE946
:102F700094E064E40E94251D8CE994E040E451EE65
:102F80006DE978E12AE030E00E94091E8CE994E0C6
:102F90006CE20E94251D8CE994E040EC51ED68E95B
:102FA0007BE12AE030E00E94091E8CE994E06CE2AB
:102FB0000E94431DBEC019821A821B821C821D8280
:102FC0001E821F82188619861A861B861C861D86FD
:102FD0001E861F86188A3AC0339434E0331609F0EF
:102FE000A8C069817A818B819C8128EE33E040E022
:102FF00050E00E94B5206F8F78A389A39AA36D81BA
:103000007E818F8198850E94B5206B8F7C8F8D8FFC
:103010009E8F89859A85AB85BC858F8B988FA98F6C
:10302000BA8F6D857E858F8598890E94B5206B014A
:103030007C0190E2C9169EE4D90690E0E90690E092
:10304000F90630F48CE162E30E941803332471C066
:10305000A0E3CA16A5E7DA06A0E0EA06A0E0FA06B1
:1030600018F48CE162E2F0CFB0E4CB16BCE9DB06E9
:10307000B0E0EB06B0E0FB0618F48CE166E2E4CFCA
:10308000E0E5CE16E3ECDE06E0E0EE06E0E0FE066C
:1030900018F48CE162E1D8CFF0E6CF16FAEEDF0645
:1030A000F0E0EF06F0E0FF0618F48CE165E1CCCF2C
:1030B00020E7C21621E1D20621E0E20620E0F20676
:1030C00018F48CE161E0C0CF30EAC31636E8D306CD
:1030D00031E0E30630E0F30618F48CE163E0B4CFAE
:1030E0008CE165E0B1CFA0ED2A2E280E49E0421513
:1030F00000F1032D10E0000F111F000F111F81E0E0
:1031000090E08C0F9D1F080F191FD8016D917D91C4
:103110008D919C912AE030E040E050E00E94B52083
:10312000620D711D811D911DF80160837183828381
:1031300093838CE994E00E94AE1F892B09F0FACEAC
:1031400081149104A104B10489F4C301B2010E9465
:10315000A90361E070E080E090E00E94A71BFFEF10
:10316000FE8B1D8A198A1A8A1B8A1C8A2F89388D20
:10317000498D5A8D82169306A406B506E0F40E9486
:10318000390329893A894B895C89280F311D411DF2
:10319000511D298B3A8B4B8B5C8B3D89381708F47A
:1031A0008D8B4E89841708F48E8B0894811C911C9A
:1031B000A11CB11C56C0C301B20128EE33E040E0AF
:1031C00050E00E94E8208CE994E0BA01A9012AE0CD
:1031D00030E00E94D71D8CE994E06CE20E94251D2E
:1031E0008CE994E06D894AE050E00E94F71D8CE97B
:1031F00094E06CE20E94251D69897A898B899C89FB
:10320000A50194010E94E8208CE994E0BA01A9018B
:103210002AE030E00E94D71D8CE994E06CE20E9425
:10322000251D8CE994E06E894AE050E00E94F71D6C
:103230008CE994E06CE20E94431D4C0C5D1C6E1CFA
:103240007F1C8B8D9C8DAD8DBE8D84159505A6053F
:10325000B70520F44F8C58A069A07AA0882499243F
:1032600054012F8D38A149A15AA1285E3340404016
:10327000504009F05ECFA296E2E10C94412180E03B
:1032800065E970E042E050E00E94AE1A0895A1E0C6
:10329000B0E0EDE4F9E10C94352180E00E94B1004A
:1032A0008DE061E00E94101C81E161E00E94101C31
:1032B0000E94210F80E060E00E94101C81E061E02C
:1032C0000E94101C8CE994E040E052EC61E070E058
:1032D0000E94271F0E94A1110E942A108CE994E0ED
:1032E00063E471E00E94661E83E793E00E94221768
:1032F0008CE994E06AE571E00E94661E8CE994E036
:1033000063E070E04AE050E00E94521E0E943F19C4
:103310007894439A86E067E00E94E716882329F0B4
:1033200043982D980E945317FBCF83E065E00E94DD
:10333000E716882329F40E94B011882309F006C1FA
:103340008CE994E062E671E00E94661E60E070E045
:1033500080E090E00E948410882349F00E94AB1125
:103360008CE994E06BE971E00E94691E2D9A0E943D
:103370001B0E22C08091E002833229F08091E3028B
:103380008B7F8093E3028091E30281FF15C082FD71
:1033900013C064EF71E080E090E00E948410882305
:1033A00059F00E94AB118CE994E06BE971E00E9446
:1033B000691E0E941B0E2D9A8091DF02823239F520
:1033C0008091E002833219F581E00E94D40D809152
:1033D000E30282FF09C08CE994E066EB71E00E9491
:1033E000691E0E94690813C064E170E080E090E00B
:1033F0000E94A71B80E2BE016F5F7F4F41E021E08A
:103400000E94E608882319F481E0809385038CE903
:1034100094E061EC71E00E94661E8FE00E94B100B2
:1034200080E00E9413041092430380E00E94230373
:103430001092010490E0983158F4292F2F5FE92F62
:10344000F0E0E051FD4F8785882311F0922FF3CFF4
:103450009093010483E08093D4020E94360F809100
:103460008503882311F00E946B0A8091E202883262
:1034700011F08A3239F48CE994E040E052EC61E0DA
:1034800070E02BC0893271F48CE994E040EA56E890
:1034900061E070E00E94271F8091C20080628093EB
:1034A000C20022C0809118038871803169F0409178
:1034B000F1025091F2026091F3027091F4024A30ED
:1034C00051056105710538F48CE994E040E855E256
:1034D00060E070E002C08CE994E00E94271F04C005
:1034E0008CE994E00E94E81F8CE994E00E94AE1FF2
:1034F000892BB1F78091E102843229F08091C100DB
:103500008F7E8093C1008091E202853259F08A3229
:1035100049F0893239F0883229F08091C100877FE3
:103520008093C1001092FF03109200041092830355
:103530000E94811B6093440370934503809346036C
:10354000909347032196E2E00C9451210E941B0EB8
:103550008091DF02823209F011CF0CCF823000F56A
:10356000E82FF0E0EE0FFF1FE95FFB4F71836083F0
:10357000882319F08130A1F408C0809169008C7F04
:10358000842B80936900E89A089580916900440F24
:10359000551F440F551F837F842B80936900E99A40
:1035A00008951F920F920FB60F9211242F933F93FD
:1035B0004F935F936F937F938F939F93AF93BF933B
:1035C000EF93FF938091070490910804892B29F0D1
:1035D000E0910704F09108040995FF91EF91BF91E4
:1035E000AF919F918F917F916F915F914F913F919B
:1035F0002F910F900FBE0F901F9018951F920F9252
:103600000FB60F9211242F933F934F935F936F93B5
:103610007F938F939F93AF93BF93EF93FF9380918B
:10362000090490910A04892B29F0E0910904F09192
:103630000A040995FF91EF91BF91AF919F918F91EE
:103640007F916F915F914F913F912F910F900FBE9E
:103650000F901F9018951F920F920FB60F92112482
:103660002F933F938F939F93AF93BF9380910F04BA
:1036700090911004A0911104B091120430911304A0
:103680000196A11DB11D232F2D5F2D3720F02D5741
:103690000196A11DB11D2093130480930F049093F4
:1036A0001004A0931104B093120480910B04909124
:1036B0000C04A0910D04B0910E040196A11DB11D42
:1036C00080930B0490930C04A0930D04B0930E040C
:1036D000BF91AF919F918F913F912F910F900FBE0E
:1036E0000F901F9018958FB7F89420910F04309188
:1036F000100440911104509112048FBFB901CA0106
:1037000008959FB7F89420910B0430910C044091D8
:103710000D0450910E0486B5A89B06C08F3F21F082
:103720002F5F3F4F4F4F5F4F9FBF542F432F322F7D
:103730002227280F311D411D511D82E0220F331F0A
:10374000441F551F8A95D1F7B901CA010895EF9218
:10375000FF920F931F93CF93DF937B018C010E9405
:10376000811BEB010EC00E94811B6C1B7D0B685EF0
:103770007340C8F30894E108F10801091109C85120
:10378000DC4FE114F1040105110569F7CDB7DEB78F
:10379000E6E00C944D21019739F0880F991F880FAE
:1037A000991F02970197F1F70895789484B5826084
:1037B00084BD84B5816084BD85B5826085BD85B5D5
:1037C000816085BDEEE6F0E0808181608083E1E884
:1037D000F0E01082808182608083808181608083BC
:1037E000E0E8F0E0808181608083E1EBF0E08081BF
:1037F00084608083E0EBF0E0808181608083EAE791
:10380000F0E0808184608083808182608083808119
:10381000816080838081806880831092C1000895D8
:10382000CF93DF93482F50E0CA0186569F4FFC018B
:1038300034914A575F4FFA018491882369F190E0EF
:10384000880F991FFC01E859FF4FA591B491FC0125
:10385000EE58FF4FC591D491662351F42FB7F894D9
:103860008C91932F909589238C93888189230BC009
:10387000623061F42FB7F8948C91932F909589233F
:103880008C938881832B88832FBF06C09FB7F894C1
:103890008C91832B8C939FBFDF91CF9108958330C0
:1038A00071F0843028F48130A1F0823021F514C009
:1038B0008630B1F08730D1F08430E9F404C08091D3
:1038C00080008F7703C0809180008F7D809380007F
:1038D000089584B58F7702C084B58F7D84BD089527
:1038E0008091B0008F778093B00008958091B000F0
:1038F0008F7D8093B0000895FF920F931F93F62E53
:10390000482F50E0CA0182559F4FFC012491CA0103
:1039100086569F4FFC0114914A575F4FFA0104915C
:103920000023C9F0222319F0822F0E944F1CE02FA0
:10393000F0E0EE0FFF1FEE58FF4FA591B4919FB737
:10394000F894FF2021F48C911095812302C08C9172
:10395000812B8C939FBF1F910F91FF9008950F9320
:103960001F93482F50E0CA0182559F4FFC012491BC
:10397000CA0186569F4FFC0104914A575F4FFA01D6
:103980001491112319F420E030E015C0222319F01E
:10399000822F0E944F1C812F90E0880F991F84581E
:1039A0009F4FFC01A591B4918C9120E030E08023E1
:1039B00011F021E030E0C9011F910F910895982F77
:1039C0008E3008F09E509770809187028295880F04
:1039D000880F807C892B80937C0080917A008064A2
:1039E00080937A0080917A0086FDFCCF2091780048
:1039F00040917900942F80E030E0282B392BC901C9
:103A00000895A0E0B0E0E7E0FDE10C942F217C01F7
:103A10006B018A01C0E0D0E00FC0D6016D916D014D
:103A2000D701ED91FC910190F081E02DC70109953E
:103A3000C80FD91F015010400115110571F7CE01B3
:103A4000CDB7DEB7E8E00C944B21DC01ED91FC91A1
:103A50000190F081E02D09950895EF92FF920F9368
:103A60001F938C016DE00E94251D7C01C8016AE056
:103A70000E94251D9C012E0D3F1DC9011F910F9114
:103A8000FF90EF900895EF92FF920F931F937C01A8
:103A90000E94251D8C01C7010E942D1D9C01200F35
:103AA000311FC9011F910F91FF90EF900895CF939F
:103AB000DF93EC016115710519F420E030E00FC0CF
:103AC000DB010D900020E9F71197A61BB70BE881E9
:103AD000F9810280F381E02DAD0109959C01C901B6
:103AE000DF91CF9108954F925F927F928F929F9234
:103AF000AF92BF92CF92DF92EF92FF920F931F93FC
:103B0000DF93CF93CDB7DEB7A1970FB6F894DEBFA2
:103B10000FBECDBF2C01742ECB01223008F42AE059
:103B200019A231E2C32ED12CCC0EDD1E822E992497
:103B3000AA24BB24672D752FA50194010E94E820BB
:103B400079018A01C801B701A50194010E94B5203D
:103B5000472D461B0894C108D1084A3010F4405D37
:103B600001C0495CF6014083E114F104010511052F
:103B700021F07E2C5F2DC801DDCFC201B6010E946D
:103B8000571DA1960FB6F894DEBF0FBECDBFCF91E3
:103B9000DF911F910F91FF90EF90DF90CF90BF903A
:103BA000AF909F908F907F905F904F900895DC0131
:103BB0002115310541F4ED91FC910190F081E02D4A
:103BC000642F099508950E94731D0895EF92FF9246
:103BD0000F931F939A017B0100E010E0B801A70149
:103BE0000E94D71D1F910F91FF90EF900895EF92C3
:103BF000FF920F931F939A01E62EFF2400E010E03E
:103C0000B801A7010E94D71D1F910F91FF90EF905F
:103C10000895A0E0B0E0EFE0FEE10C942F21EC016C
:103C20006A017B012115310541F4E881F981019098
:103C3000F081E02D642F09951BC02A303105B1F4C5
:103C400077FF13C06DE20E94251D8C014427552784
:103C5000BA014C195D096E097F09CE012AE00E9464
:103C6000731D9C01200F311F04C02AE00E94731DA8
:103C70009C01C901CDB7DEB7E8E00C944B21EF926F
:103C8000FF920F931F937B019A010027F7FC009589
:103C9000102FB801A7010E94091E1F910F91FF90DC
:103CA000EF900895EF92FF920F931F937C010E9473
:103CB0003F1E8C01C7010E942D1D9C01200F311F4A
:103CC000C9011F910F91FF90EF9008950E94571D19
:103CD0000895EF92FF920F931F937C010E94661E3E
:103CE0008C01C7010E942D1D9C01200F311FC901AD
:103CF0001F910F91FF90EF90089508951F920F92DA
:103D00000FB60F9211242F933F934F938F939F934E
:103D1000EF93FF938091C00082FD1DC04091C600CB
:103D200020915404309155042F5F3F4F2F73307012
:103D300080915604909157042817390771F0E0914B
:103D40005404F0915504EC5EFB4F408330935504CE
:103D50002093540402C08091C600FF91EF919F917F
:103D60008F914F913F912F910F900FBE0F901F9009
:103D700018951F920F920FB60F9211242F933F9315
:103D80008F939F93EF93FF93209198043091990420
:103D900080919A0490919B042817390731F48091FF
:103DA000C1008F7D8093C10014C0E0919A04F0910E
:103DB0009B04E85AFB4F208180919A0490919B04C8
:103DC00001968F73907090939B0480939A04209334
:103DD000C600FF91EF919F918F913F912F910F908E
:103DE0000FBE0F901F901895A0E0B0E0EAEFFEE143
:103DF0000C942B21FC011382128288EE93E0A0E048
:103E0000B0E084839583A683B78388EC92E09183A6
:103E100080837587648757874687318B208B138B08
:103E2000028BF58AE48AD78AC68AB18EA08E938ED9
:103E3000828E8F85848F8889858F8989868F8A89EC
:103E4000878F8B8980A32096ECE00C944721AF925A
:103E5000BF92DF92EF92FF920F931F93CF93DF9366
:103E6000EC017A018B01DD24403081EE580780E0BF
:103E7000680780E0780711F0DD24D39491E0A92E43
:103E8000B12CEC89FD89DD2069F0C50108A002C0D4
:103E9000880F991F0A94E2F7808360E079E08DE350
:103EA00090E005C0108260E874E88EE190E0A8011F
:103EB00097010E94E82021503040404050405695E4
:103EC00047953795279580E12030380720F0DD2091
:103ED00011F0DD24D6CFE889F9893083EA89FB899E
:103EE000208319A2EE89FF89408121E030E0C901D9
:103EF0000C8C02C0880F991F0A94E2F7482B40836C
:103F0000EE89FF894081C9010D8C02C0880F991F7D
:103F10000A94E2F7482B4083EE89FF894081C9016A
:103F20000E8C02C0880F991F0A94E2F7482B408339
:103F3000EE89FF8980810F8C02C0220F331F0A9403
:103F4000E2F7209528232083DF91CF911F910F91D5
:103F5000FF90EF90DF90BF90AF900895DC011C962A
:103F6000ED91FC911D97E05CFF4F21913191808193
:103F70009181281B390B2F733070C90108958CE98A
:103F800094E00E94AE1F892B11F00E947D1E0895BF
:103F9000DC011C96ED91FC911D97E05CFF4F2081A8
:103FA0003181E054F040DF01AE5BBF4F8D919C91B9
:103FB00011972817390719F42FEF3FEF07C08D919C
:103FC0009C91E80FF91F8081282F30E0C9010895E6
:103FD000DC011C96ED91FC911D97E05CFF4F208168
:103FE0003181E054F040DF01AE5BBF4F8D919C9179
:103FF00011972817390719F42FEF3FEF10C08D9153
:104000009C911197E80FF91F20818D919C91119738
:1040100001968F73907011969C938E9330E0C90136
:104020000895DC0191968C919197882339F05496EC
:10403000ED91FC915597808186FFF9CF91961C9266
:104040000895CF93DF93EC01EE85FF85E05CFF4F91
:1040500020813181E054F0402F5F3F4F2F7330704B
:10406000DF01AE5BBF4F8D919C91119728173907E7
:10407000D1F3E05CFF4F80819181E054F040E80F84
:10408000F91F6083EE85FF85E05CFF4F318320835D
:10409000EE89FF89208181E090E00F8C02C0880FBB
:1040A000991F0A94E2F7282B208381E089A3EC89E9
:1040B000FD8980818064808381E090E0DF91CF91F1
:1040C00008958F929F92AF92BF92CF92DF92EF921C
:1040D000FF920F931F9300D000D00F92EDB7FEB761
:1040E000319684E0ADB7BEB711968C9383E081839F
:1040F00087E0828385E0838381E084838CE994E098
:1041000064E174E048E554E025EC30E004EC10E0B4
:10411000B0ECEB2EF12CA1ECCA2ED12CF2ECAF2E90
:10412000B12CE6EC8E2E912C0E94F41E0F900F9075
:104130000F900F900F901F910F91FF90EF90DF90D5
:10414000CF90BF90AF909F908F900895CF93DF93C3
:104150000E94D51B0E944719CFEBDFE10E94CB12D2
:104160002097E1F30E94BF1FF9CF629FD001739F98
:10417000F001829FE00DF11D649FE00DF11D929F03
:10418000F00D839FF00D749FF00D659FF00D992742
:10419000729FB00DE11DF91F639FB00DE11DF91F66
:1041A000BD01CF0111240895AA1BBB1B51E107C01B
:1041B000AA1FBB1FA617B70710F0A61BB70B881FB7
:1041C000991F5A95A9F780959095BC01CD01089546
:1041D000A1E21A2EAA1BBB1BFD010DC0AA1FBB1F0B
:1041E000EE1FFF1FA217B307E407F50720F0A21B7D
:1041F000B30BE40BF50B661F771F881F991F1A94EA
:1042000069F760957095809590959B01AC01BD0113
:10421000CF01089597FB092E05260ED057FD04D037
:10422000D7DF0AD0001C38F4509540953095219581
:104230003F4F4F4F5F4F0895F6F7909580957095DB
:1042400061957F4F8F4F9F4F08952F923F924F92CE
:104250005F926F927F928F929F92AF92BF92CF9216
:10426000DF92EF92FF920F931F93CF93DF93CDB71F
:10427000DEB7CA1BDB0B0FB6F894DEBF0FBECDBF97
:1042800009942A88398848885F846E847D848C8468
:104290009B84AA84B984C884DF80EE80FD800C8171
:1042A0001B81AA81B981CE0FD11D0FB6F894DEBF54
:1042B0000FBECDBFED010895EE0FFF1F0590F491E5
:0842C000E02D0994F894FFCFF2
:1042C80054582074696D656F75742100576169745D
:1042D800696E672062696E640A00476F7420706BAC
:1042E800740A006461746120676F6F640A00525831
:1042F8002068616E67007363616E6E6572206D6F12
:104308006465004F70656E4C52536E67205258209A
:104318007374617274696E672000206F6E2048574D
:104328002000454550524F4D2064617461206E6FE6
:10433800742076616C6964206F722062696E6420F3
:104348006A756D70706572207365742C20666F7263
:1043580063696E672062696E640A005361766564FA
:104368002062696E64206461746120746F20454521
:1043780050524F4D0A004920616D20736C6176657B
:1043880000456E746572696E67206E6F726D616C40
:10439800206D6F646500002100270520082B092285
:1043A80009260A230A260B240C250C280C290C2A7A
:1043B800C01200001A400AA1204EA5001B1E275259
:1043C8002C23308025000005400AA1204EA500209E
:1043D800244EA52C2330004B000006400AD0009D37
:1043E80049007B289D492C233000E1000005400A44
:1043F8004501D7DC03B81E0EBF00232E48E8010094
:104408008A400A6001555502AD1E20000023C8806D
:1044180025000005400AA1204EA50020244EA52C09
:104428002330000200020002000200020002000223
:104438000002000200020002000200020002000264
:1044480000028813409C08010305060708090A0BA7
:104458000C121300010000080000200000400000BA
:1044680080010000020000040000080000100000A5
:1044780000100000200000000100000200070B0CE3
:1044880010111500000000002120011DAE1FE81FBB
:04449800C81F112008
:107E00000F92CDB7DEB7112484B714BE81FFF1D035
:107E100082E08093C00088E18093C10086E0809377
:107E2000C20080E18093C4008EE0CDD088249924E4
:107E3000CC24C394F5E0DF2EE1E1EE2E73E0F72EC3
:107E4000B6D0082F813479F4B2D08983C2D0898129
:107E5000823811F481E005C0813811F485E001C059
:107E600083E09ED09AC0823411F484E103C085344B
:107E700019F485E0B6D091C0853561F498D0082F0B
:107E800010E095D090E0982E8824802A912A880CC2
:107E9000991C82C0863521F484E0A3D080E0E1CF34
:107EA000843609F04CC083D082D0A82E80D0B82E62
:107EB00000E011E07CD0F80181938F01AE16D1F77C
:107EC00088D0FB2DF53489F4E0E0F1E00BC0F9999E
:107ED000FECF92BC81BC0894811C911C819180BD15
:107EE000FA9AF99AEA1598F358C08B2D863409F05E
:107EF00054C0F401F7BEE89507B600FCFDCFF401CD
:107F0000A0E0B1E02C9130E011968C91119790E0B7
:107F1000982F8827822B932B12960C01C7BEE895C9
:107F20001124329681E0A038B80761F7F401D7BE7A
:107F3000E89507B600FCFDCFE7BEE8952EC0843774
:107F4000F1F435D034D0182F32D0B82E42D0FB2DDA
:107F5000F63421F4F40105914F010CC0FB2DF534EA
:107F600049F4F999FECF92BC81BC0894811C911C04
:107F7000F89A00B5802F14D0115049F70EC08537FC
:107F800039F427D08EE10CD085E90AD08FE069CF93
:107F9000813511F488E017D01CD080E101D050CF9A
:107FA0009091C00095FFFCCF8093C600089580910A
:107FB000C00087FFFCCF8091C00084FD01C0A89560
:107FC0008091C6000895E0E6F0E098E19083808318
:107FD0000895EDDF803219F088E0F5DFFFCF84E10E
:107FE000DFCF1F93182FE3DF1150E9F7F2DF1F9166
:0E7FF0000895282E80E0E7DFEE27FF27099492
:027FFE0001057B
:0400000300007E007B
:00000001FF
